:10000000B0C00000CAC00000C8C00000C6C00000E8
:10001000C4C00000C2C00000C0C00000BEC00000DC
:10002000BCC00000BAC00000B8C00000B6C00000EC
:10003000B4C00000B2C00000B0C00000AEC00000FC
:10004000ACC00000AAC00000A8C00000A6C000000C
:10005000A4C00000A3C00000A0C000009EC000001B
:100060009CC000009AC0000000407A10F35A00A023
:10007000724E18090010A5D4E80000E87648170071
:1000800000E40B54020000CA9A3B000000E1F505B1
:10009000000080969800000040420F000000A086FB
:1000A00001000000102700000000E803000000002D
:1000B0006400000000000A000000000001000000D1
:1000C00000002C76D888DC674F0823DFC1DFAE59EB
:1000D000E1B1B796E5E3E453C63AE651997696E87E
:1000E000E6C28426EB898C9B62ED407C6FFCEFBC02
:1000F0009C9F40F2BAA56FA5F490055A2AF75C932D
:100100006B6CF9676DC11BFCE0E40D47FEF520E662
:10011000B500D0ED902E0300943577050080841E45
:10012000080000204E0A000000C80C333333330FA0
:10013000986E12831141EF8D2114893BE65516CF3D
:10014000FEE6DB18D1844B381BF77C1D901DA4BB49
:10015000E424203284725E228100C9F124ECA1E5FE
:100160003D2711241FBECFEFD8E0DEBFCDBF11E089
:10017000A0E0B1E0EEE7F6E102C005900D92A83AEA
:10018000B107D9F721E0A8EAB1E001C01D92A43B74
:10019000B207E1F779D10C943D0B32CF1895ECE71B
:1001A000F0E0808180648083EAE7F0E08081846011
:1001B0008083808180688083089583B7817F826097
:1001C00083BFEAE7F0E080818860808378940895B7
:1001D0002F923F924F925F926F927F928F929F9257
:1001E000AF92BF92CF92DF92EF92FF920F931F9345
:1001F000CF93DF93CDB7DEB7CE56D1090FB6F894C3
:10020000DEBF0FBECDBF982E892EAC966FAFAC97D8
:10021000AD967FAFAD97742E622E17012801C601EF
:10022000B5016E012EE5C20ED11C860123E045E02A
:10023000AF963FAFAF97AE965FAFAE97DCD45E019F
:1002400081E5A80EB11C850123E045E0C201B101A2
:10025000D2D4AE965FADAE975F937F92AF963FAD2F
:10026000AF973F936F928F929F92AD969FADAD9750
:100270009F93AC962FADAC972F9380E091E09F9326
:100280008F931F9218E21F934E0189E2880E911CF2
:100290009F928F92D0D4BF92AF92DF92CF928CE197
:1002A00091E09F938F931F921F938E010F5F1F4FBB
:1002B0001F930F93C0D4C4010DD1C8010BD10FB649
:1002C000F894DEBF0FBECDBFC259DF4F0FB6F89412
:1002D000DEBF0FBECDBFDF91CF911F910F91FF9079
:1002E000EF90DF90CF90BF90AF909F908F907F90D6
:1002F0006F905F904F903F902F9008952F923F9274
:100300004F925F926F927F928F929F92AF92BF9225
:10031000CF92DF92EF92FF920F931F93CF93DF93D1
:1003200000D000D0CDB7DEB782E090E0E5D0BC01D0
:10033000882777FD8095982FFED220E030E040E3BB
:1003400051E45ED22B013C0120E030E040E051E47A
:100350006091B0017091B1018091B2019091B301AF
:100360009ED39B01AC01C301B201E2D120E030E099
:1003700040E151E445D26093B0017093B1018093A4
:10038000B2019093B30185E090E0B6D09C838B835B
:10039000BC01882777FD8095982FCDD24B015C0159
:1003A0006091AC017091AD018091AE019091AF016F
:1003B0009B01AC01BDD19B01AC01C501B401B8D119
:1003C00020E030E040E450E41BD26093AC01709335
:1003D000AD018093AE019093AF0180E090E08CD0AE
:1003E0001C01BC01882777FD8095982FA4D26B0152
:1003F0007C016091A8017091A9018091AA0190915E
:10040000AB019B01AC0194D19B01AC01C701B601CA
:100410008FD120E030E040E450E4F2D16093A801B5
:100420007093A9018093AA019093AB01C501B40117
:100430009DD09A838983C701B60157D14C01C3016E
:10044000B2014ED15B016C01830172019401A101E3
:1004500069817A818B819C81BBDE0F900F900F9018
:100460000F90DF91CF911F910F91FF90EF90DF9050
:10047000CF90BF90AF909F908F907F906F905F9044
:100480004F903F902F9008950DD089DE96DE36DF95
:100490002FE38DE093E0215080409040E1F700C0D1
:1004A0000000F5CF1092C5008CE08093C400E0EC12
:1004B000F0E080818260808388E18093C10086E0E3
:1004C0008093C20008959091C00095FFFCCF809367
:1004D000C60008951F93CF93DF93EC0110E0FE0157
:1004E000E10FF11D8081882319F0EDDF1F5FF7CF49
:1004F000DF91CF911F91089590917C00907F982B70
:1005000090937C0020E130E080E090E0DC0143B794
:10051000416043BF889543B74E7F43BF4091780009
:1005200050917900840F951FA11DB11D21503109F3
:100530002115310561F79C01AD0182E05695479583
:10054000379527958A95D1F7A8E8B3E1D7D02CE065
:1005500096958795779567952A95D1F7695F7F4F2F
:100560008F4F9F4FE6D1B4D1CB01089520E030E00A
:1005700040EA50E445D1F6D2ABD1CB0108958F9239
:100580009F92AF92BF92CF92DF92EF92FF920F9322
:100590001F93CF93DF934B015C01EA0169016881EE
:1005A0007981882777FD8095982FC5D19B01AC0173
:1005B000C501B40121D187FF05C06A817B818C818F
:1005C0009D8181C086E08C9D80018D9D100D112440
:1005D000065011090C0F1D1FF801608171818827D9
:1005E00077FD8095982FA7D19B01AC01C501B4017F
:1005F00052D218160CF462C08E0180E090E0F1E057
:10060000CF1AD1089C012F5F3F4F79018C159D05B2
:1006100084F4F80166817781882777FD8095982F8B
:100620008AD10A5F1F4FA501940135D218160CF02C
:1006300043C086E08E9DF0018F9DF00D11248E0148
:100640000E0F1F1F3697EC0FFD1FC081D181C28096
:10065000D380E480F580BE01882777FD8095982FB0
:100660006AD19B01AC01C501B40161D04B015C01B1
:10067000A7019601F801628173818481958157D029
:100680009B01AC01C501B4010AD24B015C01F80128
:10069000608171816C1B7D0B882777FD8095982F79
:1006A0004AD19B01AC01C501B401AAD09B01AC01A8
:1006B000C701B6013DD007C0C701A4CFF8016281D0
:1006C000738184819581DF91CF911F910F91FF906C
:1006D000EF90DF90CF90BF90AF909F908F90089554
:1006E0002FE030E04DE451E04ACF26E030E049E22F
:1006F00051E045DF37D2ECD0CB01089509D0A59F5A
:10070000900DB49F900DA49F800D911D112408950C
:10071000A29FB001B39FC001A39F700D811D112442
:10072000911DB29F700D811D1124911D0895505887
:10073000BB27AA270ED075C166D130F06BD120F04F
:1007400031F49F3F11F41EF45BC10EF4E095E7FB1A
:1007500051C1E92F77D180F3BA1762077307840775
:10076000950718F071F49EF58FC10EF4E0950B2EED
:10077000BA2FA02D0B01B90190010C01CA01A001F3
:100780001124FF27591B99F0593F50F4503E68F14E
:100790001A16F040A22F232F342F4427585FF3CF8F
:1007A000469537952795A795F0405395C9F77EF460
:1007B0001F16BA0B620B730B840BBAF09150A1F0A9
:1007C000FF0FBB1F661F771F881FC2F70EC0BA0F2F
:1007D000621F731F841F48F4879577956795B795B7
:1007E000F7959E3F08F0B3CF9395880F08F09927AF
:1007F000EE0F979587950895D9D008F481E0089574
:100800000CD00FC107D140F0FED030F021F45F3F93
:1008100019F0F0C0511139C1F3C014D198F39923E4
:10082000C9F35523B1F3951B550BBB27AA276217B4
:100830007307840738F09F5F5F4F220F331F441FF9
:10084000AA1FA9F333D00E2E3AF0E0E830D0915031
:100850005040E695001CCAF729D0FE2F27D0660F1E
:10086000771F881FBB1F261737074807AB07B0E85D
:1008700009F0BB0B802DBF01FF2793585F4F2AF073
:100880009E3F510568F0B6C000C15F3FECF3983E53
:10089000DCF3869577956795B795F7959F5FC9F7D0
:1008A000880F911D9695879597F90895E1E0660F59
:1008B000771F881FBB1F621773078407BA0720F0D2
:1008C000621B730B840BBA0BEE1F88F7E09508953B
:1008D00004D06894B111D9C00895BCD088F09F5756
:1008E00090F0B92F9927B751A0F0D1F0660F771F7C
:1008F000881F991F1AF0BA95C9F712C0B13081F05C
:10090000C3D0B1E00895C0C0672F782F8827B85FA3
:1009100039F0B93FCCF3869577956795B395D9F7BC
:100920003EF490958095709561957F4F8F4F9F4FC6
:100930000895E89409C097FB3EF4909580957095D2
:1009400061957F4F8F4F9F4F9923A9F0F92F96E91B
:10095000BB279395F695879577956795B795F11190
:10096000F8CFFAF4BB0F11F460FF1BC06F5F7F4F2D
:100970008F4F9F4F16C0882311F096E911C077233F
:1009800021F09EE8872F762F05C0662371F096E848
:10099000862F70E060E02AF09A95660F771F881F17
:1009A000DAF7880F9695879597F90895990F0008BB
:1009B000550FAA0BE0E8FEEF16161706E807F90731
:1009C000C0F012161306E407F50798F0621B730BCC
:1009D000840B950B39F40A2661F0232B242B252B4D
:1009E00021F408950A2609F4A140A6958FEF811DF0
:1009F000811D089597F99F6780E870E060E0089591
:100A00009FEF80EC089500240A9416161706180626
:100A10000906089500240A94121613061406050602
:100A20000895092E0394000C11F4882352F0BB0F93
:100A300040F4BF2B11F460FF04C06F5F7F4F8F4FF6
:100A40009F4F089557FD9058440F551F59F05F3F31
:100A500071F04795880F97FB991F61F09F3F79F0E0
:100A600087950895121613061406551FF2CF469562
:100A7000F1DF08C0161617061806991FF1CF8695E4
:100A80007105610508940895E894BB2766277727C8
:100A9000CB0197F908958ADF08F48FEF08950BD002
:100AA000C0CFB1DF28F0B6DF18F0952309F0A2CF50
:100AB000A7CF1124EACFC6DFA0F3959FD1F3950FFE
:100AC00050E0551F629FF001729FBB27F00DB11DD2
:100AD000639FAA27F00DB11DAA1F649F6627B00D62
:100AE000A11D661F829F2227B00DA11D621F739F4B
:100AF000B00DA11D621F839FA00D611D221F749F59
:100B00003327A00D611D231F849F600D211D822F9F
:100B1000762F6A2F11249F5750408AF0E1F08823E6
:100B20004AF0EE0FFF1FBB1F661F771F881F9150F3
:100B30005040A9F79E3F510570F05CCFA6CF5F3FB4
:100B4000ECF3983EDCF3869577956795B795F79526
:100B5000E7959F5FC1F7FE2B880F911D96958795AE
:100B600097F9089577DFE0F09E37D8F09639B8F41A
:100B70009E3848F4672F782F8827985FF9CF86959D
:100B80007795679593959539D0F3B62FB1706B0F24
:100B9000711D811D20F4879577956795939502C007
:100BA0001CC073CF882371F4772321F09850872BD2
:100BB000762F07C0662311F499270DC09051862B1C
:100BC00070E060E02AF09A95660F771F881FDAF7C9
:100BD000880F9695879597F908959F3F31F091502A
:100BE00020F4879577956795B795880F911D969511
:100BF000879597F90895EF920F931F93CF93DF9303
:100C0000E80147FF02C034E101C034E0E42FFF27D0
:100C1000E7FDF095F7FF03C0F195E195F109E32EAB
:100C2000022F2E2FAE01F7D1CE01DF91CF911F9170
:100C30000F91EF900895AEE0B0E0E0E2F6E0F4C48A
:100C40000D891E898F89988D26E02C831A8309834C
:100C500097FF02C080E090E801979E838D83AE01EC
:100C6000455E5F4F698D7A8DCE01019611D04D8121
:100C70005E8157FD0AC02F813885421753070CF457
:100C80009A01F801E20FF31F10822E96E4E0E8C407
:100C9000ACE0B0E0EDE4F6E0B9C47C016B018A01A0
:100CA000FC0117821682838181FFB0C1CE010196BB
:100CB0004C01F7019381F60193FD859193FF81919A
:100CC0006F01882309F49EC1853239F493FD859123
:100CD00093FF81916F01853221F4B70190E006D432
:100CE000E8CF512C312C20E02032A0F48B3269F077
:100CF00030F4803259F0833269F420612CC08D3297
:100D000039F0803339F4216026C02260246023C08A
:100D1000286021C027FD27C030ED380F3A3078F425
:100D200026FF06C0FAE05F9E300D1124532E13C03B
:100D30008AE0389E300D1124332E20620CC08E3292
:100D400021F426FD5FC1206406C08C3611F42068B2
:100D500002C0883641F4F60193FD859193FF81919D
:100D60006F018111C1CF982F9F7D9554933028F446
:100D70000C5F1F4FFFE3F9830DC0833631F08337DB
:100D800071F0833509F057C021C0F8018081898353
:100D90000E5F1F4F44244394512C540114C038015A
:100DA000F2E06F0E711CF801A080B18026FF03C035
:100DB000652D70E002C06FEF7FEFC5012C878BD3EC
:100DC0002C0183012C852F77222E16C03801F2E0EA
:100DD0006F0E711CF801A080B18026FF03C0652D45
:100DE00070E002C06FEF7FEFC5012C8769D32C0143
:100DF0002C852068222E830123FC19C0832D90E0CE
:100E000048165906A0F4B70180E290E06FD33A94F7
:100E1000F5CFF50127FC859127FE81915F01B70190
:100E200090E064D331103A94F1E04F1A5108411424
:100E3000510479F7DEC0843611F0893631F5F801B6
:100E400027FF07C060817181828193810C5F1F4FF2
:100E500008C060817181882777FD8095982F0E5F8B
:100E60001F4F2F76B22E97FF09C0909580957095F1
:100E700061957F4F8F4F9F4F2068B22E2AE030E060
:100E8000A40166D3A82EA81843C0853729F42F7E65
:100E9000B22E2AE030E025C0F22FF97FBF2E8F3628
:100EA000C1F018F4883579F0ADC0803719F0883773
:100EB00021F0A8C02F2F2061B22EB4FE0DC08B2DC3
:100EC0008460B82E09C024FF0AC09F2F9660B92EF7
:100ED00006C028E030E005C020E130E002C020E19B
:100EE00032E0F801B7FE07C0608171818281938191
:100EF0000C5F1F4F06C06081718180E090E00E5F43
:100F00001F4FA40125D3A82EA818FB2DFF77BF2EB5
:100F1000B6FE0BC02B2D2E7FA51450F4B4FE0AC0D4
:100F2000B2FC08C02B2D2E7E05C07A2C2B2D03C0C1
:100F30007A2C01C0752C24FF0DC0FE01EA0DF11DB5
:100F40008081803311F4297E09C022FF06C073948A
:100F5000739404C0822F867809F0739423FD12C025
:100F600020FF06C05A2C731418F4530C5718732C16
:100F7000731460F4B70180E290E02C87B7D27394C9
:100F80002C85F6CF731410F4371801C0312C24FFD0
:100F900011C0B70180E390E02C87A8D22C8522FFF6
:100FA00016C021FF03C088E590E002C088E790E00A
:100FB000B7010CC0822F867851F021FD02C080E27B
:100FC00001C08BE227FD8DE2B70190E08FD2A5141E
:100FD00030F4B70180E390E089D25A94F8CFAA9414
:100FE000F401EA0DF11D8081B70190E07FD2A110DC
:100FF000F6CF332009F45DCEB70180E290E076D2DF
:101000003A94F7CFF7018681978102C08FEF9FEF67
:101010002C96E2E117C36F927F929F92AF92BF929C
:10102000CF92DF92EF92FF920F931F93CF93DF93B4
:10103000CDB7DEB729970FB6F894DEBF0FBECDBF90
:101040006A01B22E102F0C3320F4FF24F394F00E1B
:1010500002C04CE3F42E0F2D27E0AE014F5F5F4F2F
:1010600057D17981272F2970213031F0E1FC06C05A
:10107000E0FC06C060E005C06DE203C06BE201C0A9
:1010800060E2AE2DA07173FF36C0662311F084E0DC
:1010900001C083E08B1510F4B81A01C0B12CA11166
:1010A0000BC0F6018B2D90E2882319F091938150AB
:1010B000FBCFCB0CD11CB12C662331F0F601608341
:1010C00096012F5F3F4F6901C6010396E2FE05C0FE
:1010D0002EE4F601208331E404C02EE6F6012083DD
:1010E00031E631832283FC012B2D30E22223F1F102
:1010F00031932150FBCF72FF40C0662311F084E092
:1011000001C083E08B1510F4B81A01C0B12CA111F5
:101110000BC0F6018B2D90E2882319F0919381503A
:10112000FBCFCB0CD11CB12C662331F0F6016083D0
:1011300096012F5F3F4F6901C6010396E2FE07C08B
:1011400029E4F60120832EE4218326E406C029E663
:10115000F60120832EE6218326E62283FC012B2D37
:1011600030E2222319F031932150FBCFFC01EB0D2B
:10117000F11D10828EEF9FEFB7C0B1E0611101C089
:10118000B0E04B2F50E01816190624F49C012F5F95
:101190003F4F02C021E030E0240F351F112329F01A
:1011A000412F50E04F5F5F4F02C040E050E0420FE0
:1011B000531F2B2D30E04217530714F4B41A01C00B
:1011C000B12C2E2D287159F4F6012B2D30E222235B
:1011D00019F031932150FBCFCB0CD11CB12CBB2388
:1011E00031F0F601608396012F5F3F4F6901A11135
:1011F0000BC0F6012B2D30E3222319F0319321503F
:10120000FBCFCB0CD11CB12CF80E0A81372F3071DB
:10121000A32E74FF03C0013309F4FA941F142CF4B5
:101220002F2D293018F028E001C021E0682F392F38
:1012300097FF02C060E030E0462F532F612C712CE5
:101240003EE2932EBC01621B71099B01DC01A41BD1
:10125000B50BE1E0F0E0EC0FFD1FAE0FBF1FE12E7C
:10126000F12CF194E194F1084F3FFFEF5F0731F467
:10127000F6019082B6016F5F7F4F6B01841795076F
:101280004CF02417350734F4BD01660D771DFB01C2
:10129000118101C010E341505109FFEF6F1A7F0A1D
:1012A000B6016F5F7F4F4E155F0524F0F601108386
:1012B0006B01DACF4817590739F4063320F40533A8
:1012C00019F4A11001C011E3F6011083FB018B2D6D
:1012D00090E2882319F091938150FBCFFB01EB0D35
:1012E000F11D108280E090E029960FB6F894DEBFE1
:1012F0000FBECDBFDF91CF911F910F91FF90EF9067
:10130000DF90CF90BF90AF909F907F906F900895A7
:10131000283008F027E03327DA01990F311D87FDC7
:10132000916000966105710539F432602E5F3D933E
:1013300030E32A95E1F708959F3F30F0803871053A
:10134000610509F03C5F3C5F3D93913008F0806897
:10135000911DDF93CF931F930F93FF92EF92192F5D
:10136000987F9695E92F96959695E90FFF27EE536E
:10137000FF4F99273327EE24FF24A701E7010590AB
:101380000894079428F4360FE71EF81E491F511DD4
:10139000660F771F881F991F0694A1F70590079481
:1013A00028F4E70EF81E491F561FC11D770F881F2E
:1013B000991F661F0694A1F70590079428F4F80E6C
:1013C000491F561FC71FD11D880F991F661F771F02
:1013D0000694A1F70590079420F4490F561FC71FE4
:1013E000D81F990F661F771F881F0694A9F784914D
:1013F0001095177041F0D695C79557954795F79476
:10140000E7941A95C1F7E8E6F0E068941590159115
:1014100035916591959105907FE27395E118F10AF8
:10142000430B560BC90BD009C0F7E10CF11E431F4B
:10143000561FC91FD01D7EF4703311F48A95E6CF74
:10144000E894015030F0080F0AF40027021708F45E
:10145000202F2395022F7A3328F079E37D932A9564
:10146000E9F710C07D932A9589F6069497956795BC
:10147000379517951794E118F10A430B560BC90BD2
:10148000D00998F023957E9173957A3308F070E334
:101490007C932013B8F77E9170617D9330F0839533
:1014A00071E37D9370E32A95E1F71124EF90FF90AB
:1014B0000F911F91CF91DF91992787FD9095089506
:1014C000FC010590615070400110D8F7809590950F
:1014D0008E0F9F1F0895FC01615070400190011014
:1014E000D8F7809590958E0F9F1F08950F931F93A7
:1014F000CF93DF93182F092FEB018B8181FD03C060
:101500008FEF9FEF20C082FF10C04E815F812C8142
:101510003D81421753077CF4E881F9819F012F5FD9
:101520003F4F39832883108306C0E885F985812FD2
:101530000995892B29F72E813F812F5F3F4F3F83EC
:101540002E83812F902FDF91CF911F910F910895BE
:10155000FA01AA27283051F1203181F1E8946F93E4
:101560006E7F6E5F7F4F8F4F9F4FAF4FB1E03ED08A
:10157000B4E03CD0670F781F891F9A1FA11D680F28
:10158000791F8A1F911DA11D6A0F711D811D911D5B
:10159000A11D20D009F468943F912AE0269F1124D0
:1015A0003019305D3193DEF6CF010895462F477034
:1015B000405D4193B3E00FD0C9F7F6CF462F4F708F
:1015C000405D4A3318F0495D31FD4052419302D0ED
:1015D000A9F7EACFB4E0A695979587957795679593
:1015E000BA95C9F700976105710508959B01AC0193
:1015F0000A2E06945795479537952795BA95C9F7BA
:10160000620F731F841F951FA01D08952F923F9294
:101610004F925F926F927F928F929F92AF92BF9202
:10162000CF92DF92EF92FF920F931F93CF93DF93AE
:10163000CDB7DEB7CA1BDB0B0FB6F894DEBF0FBE0B
:10164000CDBF09942A88398848885F846E847D8458
:101650008C849B84AA84B984C884DF80EE80FD805A
:101660000C811B81AA81B981CE0FD11D0FB6F894D0
:0E167000DEBF0FBECDBFED010895F894FFCF91
:10167E005469202533642043202564202020546F94
:10168E002025336420432025640D0A004C20257349
:10169E002020282573290D0A00C7FF000048C2C765
:1016AE0001000000007B050000C842D80800004879
:1016BE0043E70B00009643B20E0000C8430400003F
:1016CE0000004005003333F33F06006666E63F0830
:1016DE00009A99D93F0A00CDCCCC3F0C000000C037
:1016EE003F0F003333B33F14006666A63F1C009ACB
:1016FE0099993F2800CDCC8C3F44003333833F90E3
:10170E00010000803F200348E17A3F5C0366666675
:08171E003F7003CDCC4C3F00ED
:00000001FF
